******************************************************************************
               TMS320C6x Linker PC v7.2.1                      
******************************************************************************
>> Linked Thu May 24 22:14:47 2012

OUTPUT FILE NAME:   <KeyStone_Multicore_Navigator.out>
ENTRY POINT SYMBOL: "_c_int00"  address: 0c06e180


MEMORY CONFIGURATION

         name            origin    length      used     unused   attr    fill
----------------------  --------  ---------  --------  --------  ----  --------
  VECTORS               00800000   00000200  00000200  00000000  RWIX
  LL2_RW_DATA           00800200   0003fe00  0003d3b8  00002a48  RWIX
  SL2                   0c000000   00200000  0007c9b4  0018364c  RWIX
  DDR3_CODE             80000000   01000000  00000000  01000000  RWIX
  DDR3_R_DATA           81000000   01000000  00000000  01000000  RWIX
  DDR3_RW_DATA          82000000   06000000  04240000  01dc0000  RWIX


SEGMENT ALLOCATION MAP

run origin  load origin   length   init length attrs members
----------  ----------- ---------- ----------- ----- -------
00800000    00800000    00000200   00000200    r-x
  00800000    00800000    00000200   00000200    r-x vecs
00800200    00800200    0003ca20   00000000    rw-
  00800200    00800200    0001e000   00000000    rw- PacketData.buffer_LL2
  0081e200    0081e200    00018080   00000000    rw- QMSS_Data.Descriptor_LL2
  00836280    00836280    000051a0   00000000    rw- .far
  0083b420    0083b420    00001000   00000000    rw- .stack
  0083c420    0083c420    00000800   00000000    rw- .sysmem
0083cc20    0083cc20    000008c8   000007a8    rw-
  0083cc20    0083cc20    000007a8   000007a8    rw- .fardata
  0083d3c8    0083d3c8    00000120   00000000    rw- .cio
0083d4e8    0083d4e8    000000d0   000000b8    rw-
  0083d4e8    0083d4e8    000000b8   000000b8    rw- .neardata
  0083d5a0    0083d5a0    00000018   00000000    rw- .bss
0c000000    0c000000    00060080   00000000    rw-
  0c000000    0c000000    00040000   00000000    rw- PacketData.buffer_SL2
  0c040000    0c040000    00020080   00000000    rw- QMSS_Data.Descriptor_SL2
0c060080    0c060080    0000e760   0000e760    r-x
  0c060080    0c060080    0000e760   0000e760    r-x .text
0c06e7e0    0c06e7e0    0000c500   00000000    rw-
  0c06e7e0    0c06e7e0    0000c500   00000000    rw- QMSS_Data.linkingRAM1
0c07ace0    0c07ace0    00001cd4   00001cd4    r--
  0c07ace0    0c07ace0    00001658   00001658    r-- .const
  0c07c338    0c07c338    0000067c   0000067c    r-- .cinit
82000000    82000000    04240000   00000000    rw-
  82000000    82000000    04060000   00000000    rw- QMSS_Data.Descriptor_DDR
  86060000    86060000    001e0000   00000000    rw- PacketData.buffer_DDR


SECTION ALLOCATION MAP

 output                                  attributes/
section   page    origin      length       input sections
--------  ----  ----------  ----------   ----------------
vecs       0    00800000    00000200     
                  00800000    00000200     MNav_vectors.obj (vecs)

PacketData.buffer_LL2 
*          0    00800200    0001e000     UNINITIALIZED
                  00800200    0001e000     MNav_Init.obj (PacketData.buffer_LL2)

QMSS_Data.Descriptor_LL2 
*          0    0081e200    00018080     UNINITIALIZED
                  0081e200    00018080     MNav_Init.obj (QMSS_Data.Descriptor_LL2)

.far       0    00836280    000051a0     UNINITIALIZED
                  00836280    00005018     MNav_Test.obj (.far)
                  0083b298    00000008     --HOLE--
                  0083b2a0    000000d8     rts6600e_elf.lib : trgdrv.obj (.far)
                  0083b378    00000008     --HOLE--
                  0083b380    000000a0                      : defs.obj (.far)

.stack     0    0083b420    00001000     UNINITIALIZED
                  0083b420    00000008     rts6600e_elf.lib : boot.obj (.stack)
                  0083b428    00000ff8     --HOLE--

.sysmem    0    0083c420    00000800     UNINITIALIZED
                  0083c420    00000008     rts6600e_elf.lib : memory.obj (.sysmem)
                  0083c428    000007f8     --HOLE--

.fardata   0    0083cc20    000007a8     
                  0083cc20    000002d0     MNav_Init.obj (.fardata:freeHostQueueCfgTable)
                  0083cef0    00000150     MNav_Init.obj (.fardata:flowCfgTable)
                  0083d040    000000f0     rts6600e_elf.lib : defs.obj (.fardata:_ftable)
                  0083d130    00000090     MNav_Init.obj (.fardata:descMemRegionsCfg)
                  0083d1c0    00000078     rts6600e_elf.lib : lowlev.obj (.fardata:_device)
                  0083d238    00000008                      : _lock.obj (.fardata)
                  0083d240    00000070     MNav_Init.obj (.fardata:freeMonoQueueCfgTable)
                  0083d2b0    00000050     MNav_Test.obj (.fardata)
                  0083d300    00000050     rts6600e_elf.lib : lowlev.obj (.fardata:_stream)
                  0083d350    00000024     KeyStone_common.obj (.fardata:timerRegs)
                  0083d374    0000000c     rts6600e_elf.lib : exit.obj (.fardata)
                  0083d380    00000010     KeyStone_common.obj (.fardata:mem_prot_key)
                  0083d390    0000000c     rts6600e_elf.lib : memory.obj (.fardata)
                  0083d39c    00000004                      : defs.obj (.fardata)
                  0083d3a0    00000008     KeyStone_Navigator_init_drv.obj (.fardata:qmPdspCmd)
                  0083d3a8    00000008     --HOLE--
                  0083d3b0    00000008     KeyStone_Navigator_init_drv.obj (.fardata:qmPdspCtrlRegs)
                  0083d3b8    00000008     --HOLE--
                  0083d3c0    00000008     KeyStone_Navigator_init_drv.obj (.fardata:qmPdspIRam)

.cio       0    0083d3c8    00000120     UNINITIALIZED
                  0083d3c8    00000120     rts6600e_elf.lib : trgmsg.obj (.cio)

.neardata 
*          0    0083d4e8    000000b8     
                  0083d4e8    00000064     KeyStone_Navigator_init_drv.obj (.neardata)
                  0083d54c    00000050     KeyStone_common.obj (.neardata)
                  0083d59c    00000004     KeyStone_DDR_Init.obj (.neardata)

.rodata    0    0083d5a0    00000000     UNINITIALIZED

.bss       0    0083d5a0    00000018     UNINITIALIZED
                  0083d5a0    00000010     MNav_Init.obj (.bss)
                  0083d5b0    00000004     MNav_QM_Intc_setup.obj (.bss)
                  0083d5b4    00000004     MNav_Test.obj (.bss)

PacketData.buffer_SL2 
*          0    0c000000    00040000     UNINITIALIZED
                  0c000000    00040000     MNav_Init.obj (PacketData.buffer_SL2)

QMSS_Data.Descriptor_SL2 
*          0    0c040000    00020080     UNINITIALIZED
                  0c040000    00020080     MNav_Init.obj (QMSS_Data.Descriptor_SL2)

.text      0    0c060080    0000e760     
                  0c060080    00002800     KeyStone_DDR_Init.obj (.text)
                  0c062880    00001c40     KeyStone_common.obj (.text)
                  0c0644c0    00001b20     KeyStone_Navigator_init_drv.obj (.text)
                  0c065fe0    00000f20     MNav_Test.obj (.text)
                  0c066f00    000007e0     MNav_Test_main.obj (.text)
                  0c0676e0    000005e0     rts6600e_elf.lib : divd.obj (.text:__c6xabi_divd)
                  0c067cc0    000005c0                      : _printfi.obj (.text:_getarg_diouxp)
                  0c068280    00000500     MNav_Init.obj (.text)
                  0c068780    000004a0     rts6600e_elf.lib : _printfi.obj (.text:_setfield)
                  0c068c20    00000480                      : _printfi.obj (.text:_printfi)
                  0c0690a0    000003e0     MNav_Test.obj (.text:retain)
                  0c069480    000003a0     rts6600e_elf.lib : divf.obj (.text:__c6xabi_divf)
                  0c069820    00000300                      : fputs.obj (.text:fputs)
                  0c069b20    000002e0                      : _printfi.obj (.text:_pproc_fwp)
                  0c069e00    000002c0                      : _printfi.obj (.text:_pproc_fge)
                  0c06a0c0    000002a0                      : _printfi.obj (.text:fcvt)
                  0c06a360    00000280     MNav_QM_Intc_setup.obj (.text)
                  0c06a5e0    00000280     rts6600e_elf.lib : _printfi.obj (.text:ecvt)
                  0c06a860    00000280                      : memory.obj (.text:free)
                  0c06aae0    00000240                      : imath64.obj (.text:__c6xabi_divull)
                  0c06ad20    00000240                      : _printfi.obj (.text:_pconv_e)
                  0c06af60    00000220                      : _printfi.obj (.text:_pproc_diouxp)
                  0c06b180    00000220                      : _printfi.obj (.text:_pproc_str)
                  0c06b3a0    00000200                      : _printfi.obj (.text:_pconv_g)
                  0c06b5a0    000001c0                      : _printfi.obj (.text:_mcpy)
                  0c06b760    000001a0                      : trgdrv.obj (.text:HOSTrename)
                  0c06b900    000001a0                      : imath40.obj (.text:__c6xabi_divul)
                  0c06baa0    000001a0                      : memory.obj (.text:malloc)
                  0c06bc40    000001a0                      : setvbuf.obj (.text:setvbuf)
                  0c06bde0    00000180                      : copy_decompress_rle.obj (.text:__TI_decompress_rle_core)
                  0c06bf60    00000180                      : autoinit.obj (.text:_auto_init_elf)
                  0c06c0e0    00000180     KeyStone_common.obj (.text:retain)
                  0c06c260    00000160     rts6600e_elf.lib : frcmpyd_div.obj (.text:__c6xabi_frcmpyd_div)
                  0c06c3c0    00000140                      : _printfi.obj (.text:_pproc_fflags)
                  0c06c500    00000140                      : fputc.obj (.text:fputc)
                  0c06c640    00000140                      : lowlev.obj (.text:getdevice)
                  0c06c780    00000120                      : _printfi.obj (.text:_ltostr)
                  0c06c8a0    00000120                      : fclose.obj (.text:fclose)
                  0c06c9c0    00000100                      : trgdrv.obj (.text:HOSTlseek)
                  0c06cac0    00000100                      : _io_perm.obj (.text:_wrt_ok)
                  0c06cbc0    00000100                      : cpy_tbl.obj (.text:copy_in)
                  0c06ccc0    000000e0                      : trgdrv.obj (.text:HOSTopen)
                  0c06cda0    000000e0                      : _printfi.obj (.text:_div)
                  0c06ce80    000000e0                      : atoi.obj (.text:atoi)
                  0c06cf60    000000e0                      : lowlev.obj (.text:close)
                  0c06d040    000000e0                      : copy_zero_init.obj (.text:decompress:ZI:__TI_zero_init)
                  0c06d120    000000e0                      : exit.obj (.text:exit)
                  0c06d200    000000e0                      : memset.obj (.text:memset)
                  0c06d2e0    000000c0                      : trgdrv.obj (.text:HOSTread)
                  0c06d3a0    000000c0                      : trgdrv.obj (.text:HOSTunlink)
                  0c06d460    000000c0                      : trgdrv.obj (.text:HOSTwrite)
                  0c06d520    000000c0                      : divu.obj (.text:__divu)
                  0c06d5e0    000000c0                      : fopen.obj (.text:_cleanup)
                  0c06d6a0    000000c0                      : fflush.obj (.text:_doflush)
                  0c06d760    000000c0                      : fseek.obj (.text:fseek)
                  0c06d820    000000c0                      : lowlev.obj (.text:lseek)
                  0c06d8e0    000000c0                      : ltoa.obj (.text:ltoa)
                  0c06d9a0    000000c0                      : lowlev.obj (.text:write)
                  0c06da60    000000a0                      : trgdrv.obj (.text:HOSTclose)
                  0c06db00    000000a0                      : frcmpyf_div.obj (.text:__c6xabi_frcmpyf_div)
                  0c06dba0    000000a0                      : _printfi.obj (.text:_ecpy)
                  0c06dc40    000000a0                      : _printfi.obj (.text:_fcpy)
                  0c06dce0    000000a0                      : _printfi.obj (.text:_pconv_f)
                  0c06dd80    000000a0                      : lowlev.obj (.text:finddevice)
                  0c06de20    000000a0                      : memcpy64.obj (.text:memcpy)
                  0c06dec0    000000a0                      : memory.obj (.text:minsert)
                  0c06df60    000000a0                      : memory.obj (.text:mremove)
                  0c06e000    00000080                      : fixdu.obj (.text:__c6xabi_fixdu)
                  0c06e080    00000080                      : fixfu.obj (.text:__c6xabi_fixfu)
                  0c06e100    00000080                      : llshift.obj (.text:__c6xabi_llshl)
                  0c06e180    00000080                      : boot.obj (.text:_c_int00)
                  0c06e200    00000080                      : memory.obj (.text:_minit)
                  0c06e280    00000080                      : printf.obj (.text:printf)
                  0c06e300    00000080                      : trgmsg.obj (.text:readmsg)
                  0c06e380    00000080                      : lowlev.obj (.text:unlink)
                  0c06e400    00000060                      : llshift.obj (.text:__c6xabi_llshru)
                  0c06e460    00000060                      : imath64.obj (.text:_subcull)
                  0c06e4c0    00000060                      : memccpy.obj (.text:memccpy)
                  0c06e520    00000060                      : trgmsg.obj (.text:writemsg)
                  0c06e580    00000040                      : isinf.obj (.text:__c6xabi_isinf)
                  0c06e5c0    00000040                      : _printfi.obj (.text:__c6xabi_isnan)
                  0c06e600    00000040                      : divd.obj (.text:__c6xabi_isnan)
                  0c06e640    00000040                      : args_main.obj (.text:_args_main)
                  0c06e680    00000040                      : fputs.obj (.text:puts)
                  0c06e6c0    00000020                      : divf.obj (.text:__c6xabi_isnanf)
                  0c06e6e0    00000020                      : negll.obj (.text:__c6xabi_negll)
                  0c06e700    00000020                      : tdeh_init.obj (.text:__tdeh_init)
                  0c06e720    00000020                      : _lock.obj (.text:_nop)
                  0c06e740    00000020                      : printf.obj (.text:_outc)
                  0c06e760    00000020                      : printf.obj (.text:_outs)
                  0c06e780    00000020                      : exit.obj (.text:abort)
                  0c06e7a0    00000020                      : copy_decompress_none.obj (.text:decompress:none:__TI_decompress_none)
                  0c06e7c0    00000020                      : copy_decompress_rle.obj (.text:decompress:rle24:__TI_decompress_rle24)

QMSS_Data.linkingRAM1 
*          0    0c06e7e0    0000c500     UNINITIALIZED
                  0c06e7e0    0000c500     MNav_Init.obj (QMSS_Data.linkingRAM1)

.const     0    0c07ace0    00001658     
                  0c07ace0    000005d4     MNav_Init.obj (.const:acc48_be)
                  0c07b2b4    000004b8     KeyStone_common.obj (.const:.string)
                  0c07b76c    0000040c     MNav_Test.obj (.const:.string)
                  0c07bb78    000003cc     MNav_Test_main.obj (.const:.string)
                  0c07bf44    000001c0     KeyStone_Navigator_init_drv.obj (.const:.string)
                  0c07c104    00000002     rts6600e_elf.lib : fputs.obj (.const:.string)
                  0c07c106    0000000a     --HOLE-- [fill = 0]
                  0c07c110    00000101                      : ctype.obj (.const:_ctypes_)
                  0c07c211    00000003     --HOLE-- [fill = 0]
                  0c07c214    0000008c     MNav_Init.obj (.const:.string)
                  0c07c2a0    00000044     KeyStone_DDR_Init.obj (.const:.string)
                  0c07c2e4    00000023     rts6600e_elf.lib : _printfi.obj (.const:.string)
                  0c07c307    00000001     --HOLE-- [fill = 0]
                  0c07c308    00000014     MNav_QM_Intc_setup.obj (.const:.string)
                  0c07c31c    00000004     --HOLE-- [fill = 0]
                  0c07c320    00000008     rts6600e_elf.lib : divd.obj (.const:initial_approx$1)
                  0c07c328    00000008     --HOLE-- [fill = 0]
                  0c07c330    00000008                      : divf.obj (.const:initial_approx$1)

.cinit     0    0c07c338    0000067c     
                  0c07c338    00000514     (.cinit..fardata.load) [load image, compression = rle]
                  0c07c84c    000000ba     (.cinit..neardata.load) [load image, compression = rle]
                  0c07c906    00000002     --HOLE-- [fill = 0]
                  0c07c908    0000000c     (__TI_handler_table)
                  0c07c914    00000008     (.cinit..bss.load) [load image, compression = zero_init]
                  0c07c91c    00000008     (.cinit..far.load) [load image, compression = zero_init]
                  0c07c924    00000008     (.cinit.PacketData.buffer_DDR.load) [load image, compression = zero_init]
                  0c07c92c    00000008     (.cinit.PacketData.buffer_LL2.load) [load image, compression = zero_init]
                  0c07c934    00000008     (.cinit.PacketData.buffer_SL2.load) [load image, compression = zero_init]
                  0c07c93c    00000008     (.cinit.QMSS_Data.Descriptor_DDR.load) [load image, compression = zero_init]
                  0c07c944    00000008     (.cinit.QMSS_Data.Descriptor_LL2.load) [load image, compression = zero_init]
                  0c07c94c    00000008     (.cinit.QMSS_Data.Descriptor_SL2.load) [load image, compression = zero_init]
                  0c07c954    00000008     (.cinit.QMSS_Data.linkingRAM1.load) [load image, compression = zero_init]
                  0c07c95c    00000058     (__TI_cinit_table)

QMSS_Data.Descriptor_DDR 
*          0    82000000    04060000     UNINITIALIZED
                  82000000    04060000     MNav_Init.obj (QMSS_Data.Descriptor_DDR)

PacketData.buffer_DDR 
*          0    86060000    001e0000     UNINITIALIZED
                  86060000    001e0000     MNav_Init.obj (PacketData.buffer_DDR)


LINKER GENERATED COPY TABLES

__TI_cinit_table @ 0c07c95c records: 11, size/record: 8, table size: 88
	.fardata: load addr=0c07c338, load size=00000514 bytes, run addr=0083cc20, run size=000007a8 bytes, compression=rle
	.neardata: load addr=0c07c84c, load size=000000ba bytes, run addr=0083d4e8, run size=000000b8 bytes, compression=rle
	.bss: load addr=0c07c914, load size=00000008 bytes, run addr=0083d5a0, run size=00000018 bytes, compression=zero_init
	.far: load addr=0c07c91c, load size=00000008 bytes, run addr=00836280, run size=000051a0 bytes, compression=zero_init
	PacketData.buffer_DDR: load addr=0c07c924, load size=00000008 bytes, run addr=86060000, run size=001e0000 bytes, compression=zero_init
	PacketData.buffer_LL2: load addr=0c07c92c, load size=00000008 bytes, run addr=00800200, run size=0001e000 bytes, compression=zero_init
	PacketData.buffer_SL2: load addr=0c07c934, load size=00000008 bytes, run addr=0c000000, run size=00040000 bytes, compression=zero_init
	QMSS_Data.Descriptor_DDR: load addr=0c07c93c, load size=00000008 bytes, run addr=82000000, run size=04060000 bytes, compression=zero_init
	QMSS_Data.Descriptor_LL2: load addr=0c07c944, load size=00000008 bytes, run addr=0081e200, run size=00018080 bytes, compression=zero_init
	QMSS_Data.Descriptor_SL2: load addr=0c07c94c, load size=00000008 bytes, run addr=0c040000, run size=00020080 bytes, compression=zero_init
	QMSS_Data.linkingRAM1: load addr=0c07c954, load size=00000008 bytes, run addr=0c06e7e0, run size=0000c500 bytes, compression=zero_init


LINKER GENERATED HANDLER TABLE

__TI_handler_table @ 0c07c908 records: 3, size/record: 4, table size: 12
	index: 0, handler: __TI_decompress_rle24
	index: 1, handler: __TI_decompress_none
	index: 2, handler: __TI_zero_init


GLOBAL SYMBOLS: SORTED ALPHABETICALLY BY Name 

address    name
--------   ----
0c06e780   C$$EXIT
0c06e578   C$$IO$$
0083d550   CGEM_regs
0c06a42c   CP_INTC_Init_QM
0083d59c   DDR_Regs
0c067294   DSPCoreAccessQueueTest
0c0641b8   EXC_external
0c064398   EXC_internal
0c064484   EXC_nmi
0c0644a0   EXC_swgen
0c063f70   Exception_cfg
0c06c0e0   Exeception_ISR
0c06da60   HOSTclose
0c06c9c0   HOSTlseek
0c06ccc0   HOSTopen
0c06d2e0   HOSTread
0c06b760   HOSTrename
0c06d3a0   HOSTunlink
0c06d460   HOSTwrite
0c064ff8   KeyStone_Copy_FDQ
0c062e48   KeyStone_DDR_PLL_init
0c064b78   KeyStone_Host_Descriptor_Queues_init
0c0632f4   KeyStone_L1_cfg
0c0633f0   KeyStone_L2_cfg
0c064e28   KeyStone_Mono_Descriptor_Queues_init
0c062fcc   KeyStone_PA_PLL_init
0c0647a8   KeyStone_QMSS_Descriptor_Regions_init
0c0646d8   KeyStone_QMSS_Linking_RAM_init
0c065288   KeyStone_Qmss_Config_Acc_Channel
0c0655b0   KeyStone_Qmss_Config_Reclaim_Queue
0c0650c4   KeyStone_Qmss_Download_Firmware
0c065544   KeyStone_Qmss_config_Acc_Timer
0c065478   KeyStone_Qmss_disable_Acc_Channel
0c06322c   KeyStone_XM_cfg
0c062ab8   KeyStone_main_PLL_init
0c065618   KeyStone_pktDma_Global_Control
0c065680   KeyStone_pktDma_TxCh_config
0c0656d8   KeyStone_pktDma_configureRxFlow
0c063aec   Keystone_disable_PSC_Power_Domain
0c063a98   Keystone_disable_PSC_module
0c063a34   Keystone_enable_PSC_module
0c068380   PktDMA_init
0c067374   PktDmaTest
0c0668f0   PktDmaThroughput
0c067320   PktDmaThroughputTest
0c0682c0   QMSS_init
0c06a538   QM_Interrupts_Init
0c0690a0   QueueAccumulationISR
0c069430   QueuePendISR
0c0672d0   QueuePendInterruptTest
0c066354   QueuePopCycleTest
0c0661f0   QueuePushCycleTest
0c067058   QueuePushPopTest
0c066568   QueuePushToAccumulationDelayTest
0c0667a0   QueuePushToPendInterruptDelayTest
0c066490   QueuePushToPopDelayTest
0c06680c   QueueReclamationDelayTest
0c063b40   Reset_Timer
0c063e14   Service_Watchdog
0c060194   TCI6608_EVM_DDR_Init
0c061e14   TCI6614_Huawei_DDR_Init
0c0613d0   TCI6614_VDB_DDR_Init
0c0609d4   TCI6618_EVM_DDR_Init
0c063ecc   TSC_delay_ms
0c063f28   TSC_delay_us
0c063eb0   TSC_init
0c063b88   Timer_Init
0c063c50   Timer_One_Shot_Init
0c063d18   Watchdog_Timer_Init
0083d54c   XMC_regs
0083d3c8   __CIOBUF_
0c07c95c   __TI_CINIT_Base
0c07c9b4   __TI_CINIT_Limit
0c07c908   __TI_Handler_Table_Base
0c07c914   __TI_Handler_Table_Limit
0083c420   __TI_STACK_END
00001000   __TI_STACK_SIZE
0083d4e8   __TI_STATIC_BASE
00000800   __TI_SYSMEM_SIZE
00000001   __TI_args_main
0c06e7a0   __TI_decompress_none
0c06e7c0   __TI_decompress_rle24
0083d37c   __TI_enable_exit_profile_output
ffffffff   __TI_pprof_out_hndl
ffffffff   __TI_prof_data_size
ffffffff   __TI_prof_data_start
0c06d040   __TI_zero_init
ffffffff   __binit__
0c0676e0   __c6xabi_divd
0c069480   __c6xabi_divf
0c06d520   __c6xabi_divu
0c06b900   __c6xabi_divul
0c06aae0   __c6xabi_divull
0c06e000   __c6xabi_fixdu
0c06e080   __c6xabi_fixfu
0c06c260   __c6xabi_frcmpyd_div
0c06db00   __c6xabi_frcmpyf_div
0c06e580   __c6xabi_isinf
0c06e100   __c6xabi_llshl
0c06e400   __c6xabi_llshru
0c06e6e0   __c6xabi_negll
ffffffff   __c_args__
0c06d520   __divu
0c06e700   __tdeh_init
0c06e640   _args_main
0c06bf60   _auto_init_elf
0c06e180   _c_int00
0c06d5e0   _cleanup
0083d374   _cleanup_ptr
0c07c110   _ctypes_
0c06d6a0   _doflush
0083d378   _dtors_ptr
0083d39c   _ft_end
0083d040   _ftable
0083d238   _lock
0c06e200   _minit
0c06e720   _nop
0c068c20   _printfi
0083b420   _stack
0c06e460   _subcull
0083c420   _sys_memory
0083b380   _tmpnams
0083d23c   _unlock
0c06cac0   _wrt_ok
0c06e780   abort
0c07ace0   acc48_be
0c06ce80   atoi
ffffffff   binit
0083d554   boot_cfg_regs
0c063e58   calc_cycle_measure_overhead
0c068498   checkQueues
0c06cf60   close
0c06cbc0   copy_in
0083d558   cpIntc0Regs
0083d55c   cpIntc1Regs
0083d598   cycle_measure_overhead
0083d130   descMemRegionsCfg
0c0635c4   edma_Init
0c06d120   exit
0c06c8a0   fclose
0083cef0   flowCfgTable
0c06c500   fputc
0c069820   fputs
0c06a860   free
0083cc20   freeHostQueueCfgTable
0083d240   freeMonoQueueCfgTable
0c06d760   fseek
0083d568   gEDMACC0Regs
0083d56c   gEDMACC1Regs
0083d570   gEDMACC2Regs
0083d2b0   hiQuAccCfg
82000000   hostDescriptor_DDR
0081e200   hostDescriptor_LL2
0c040000   hostDescriptor_SL2
0083d5b4   intTSCL
0c06e7e0   linkingRAM1
0083d2d8   loQuAccCfg
0c063098   lock_mem_prot_regs
0c06d820   lseek
0c06d8e0   ltoa
0c067500   main
0c06baa0   malloc
0083d380   mem_prot_key
0c06e4c0   memccpy
0c06de20   memcpy
0c0640cc   memory_protection_exception
0c06d200   memset
82040000   monoDescriptor_DDR
00826200   monoDescriptor_LL2
0c050000   monoDescriptor_SL2
0083d548   numLinkingEntry
0083d534   paDmaCfgRegs
0083d53c   paDmaRxChCfgRegs
0083d544   paDmaRxFlowCfgRegs
0083d538   paDmaTxChCfgRegs
0083d540   paDmaTxChPriority
86060000   packetBuffer_DDR_Size0
86080000   packetBuffer_DDR_Size1
860c0000   packetBuffer_DDR_Size2
86140000   packetBuffer_DDR_Size3
00800200   packetBuffer_LL2_Size0
00802200   packetBuffer_LL2_Size1
00806200   packetBuffer_LL2_Size2
0080e200   packetBuffer_LL2_Size3
0c000000   packetBuffer_SL2_Size0
0c010000   packetBuffer_SL2_Size1
0c020000   packetBuffer_SL2_Size2
0c030000   packetBuffer_SL2_Size3
0083d560   pllc_regs
0c06e280   printf
0083d564   pscRegs
0c06c500   putc
0c06e680   puts
0083d4e8   qmCfgRegs
0083d4ec   qmDescriptorRegions
0083d50c   qmDmaCfgRegs
0083d514   qmDmaRxChCfgRegs
0083d51c   qmDmaRxFlowCfgRegs
0083d510   qmDmaTxChCfgRegs
0083d518   qmDmaTxChPriority
0083d508   qmIntRegs
0083d3a0   qmPdspCmd
0083d3b0   qmPdspCtrlRegs
0083d3c0   qmPdspIRam
0083d4f8   queueManageData
0083d4fc   queueManageProxyData
0083d4f4   queueManageProxyRegs
0083d4f0   queueManageRegs
0083d500   queueStatusConfigRegs
0083d504   queueThresholdStatus
0c06e300   readmsg
0c06e380   remove
0c06bc40   setvbuf
0083d520   srioDmaCfgRegs
0083d528   srioDmaRxChCfgRegs
0083d530   srioDmaRxFlowCfgRegs
0083d524   srioDmaTxChCfgRegs
0083d52c   srioDmaTxChPriority
0083d574   timer0Regs
0083d578   timer1Regs
0083d57c   timer2Regs
0083d580   timer3Regs
0083d584   timer4Regs
0083d588   timer5Regs
0083d58c   timer6Regs
0083d590   timer7Regs
0083d594   timer8Regs
0083d350   timerRegs
0083d5a4   uiInitialHostFdqNum
0083d5a8   uiInitialMonoFdqNum
0083d5b0   uiQ662_pend_event_num
0083d5a0   uiUsedDescRegionNum
0083d5ac   uiUsedRxFlowNum
00836280   uiaDescriptorBuffer
00837280   uiaDescriptorPintPongBufferHi
00839290   uiaDescriptorPintPongBufferLo
0c06e380   unlink
0c063164   unlock_mem_prot_regs
00800000   vectors
0c06d9a0   write
0c06e520   writemsg


GLOBAL SYMBOLS: SORTED BY Symbol Address 

address    name
--------   ----
00000001   __TI_args_main
00000800   __TI_SYSMEM_SIZE
00001000   __TI_STACK_SIZE
00800000   vectors
00800200   packetBuffer_LL2_Size0
00802200   packetBuffer_LL2_Size1
00806200   packetBuffer_LL2_Size2
0080e200   packetBuffer_LL2_Size3
0081e200   hostDescriptor_LL2
00826200   monoDescriptor_LL2
00836280   uiaDescriptorBuffer
00837280   uiaDescriptorPintPongBufferHi
00839290   uiaDescriptorPintPongBufferLo
0083b380   _tmpnams
0083b420   _stack
0083c420   __TI_STACK_END
0083c420   _sys_memory
0083cc20   freeHostQueueCfgTable
0083cef0   flowCfgTable
0083d040   _ftable
0083d130   descMemRegionsCfg
0083d238   _lock
0083d23c   _unlock
0083d240   freeMonoQueueCfgTable
0083d2b0   hiQuAccCfg
0083d2d8   loQuAccCfg
0083d350   timerRegs
0083d374   _cleanup_ptr
0083d378   _dtors_ptr
0083d37c   __TI_enable_exit_profile_output
0083d380   mem_prot_key
0083d39c   _ft_end
0083d3a0   qmPdspCmd
0083d3b0   qmPdspCtrlRegs
0083d3c0   qmPdspIRam
0083d3c8   __CIOBUF_
0083d4e8   __TI_STATIC_BASE
0083d4e8   qmCfgRegs
0083d4ec   qmDescriptorRegions
0083d4f0   queueManageRegs
0083d4f4   queueManageProxyRegs
0083d4f8   queueManageData
0083d4fc   queueManageProxyData
0083d500   queueStatusConfigRegs
0083d504   queueThresholdStatus
0083d508   qmIntRegs
0083d50c   qmDmaCfgRegs
0083d510   qmDmaTxChCfgRegs
0083d514   qmDmaRxChCfgRegs
0083d518   qmDmaTxChPriority
0083d51c   qmDmaRxFlowCfgRegs
0083d520   srioDmaCfgRegs
0083d524   srioDmaTxChCfgRegs
0083d528   srioDmaRxChCfgRegs
0083d52c   srioDmaTxChPriority
0083d530   srioDmaRxFlowCfgRegs
0083d534   paDmaCfgRegs
0083d538   paDmaTxChCfgRegs
0083d53c   paDmaRxChCfgRegs
0083d540   paDmaTxChPriority
0083d544   paDmaRxFlowCfgRegs
0083d548   numLinkingEntry
0083d54c   XMC_regs
0083d550   CGEM_regs
0083d554   boot_cfg_regs
0083d558   cpIntc0Regs
0083d55c   cpIntc1Regs
0083d560   pllc_regs
0083d564   pscRegs
0083d568   gEDMACC0Regs
0083d56c   gEDMACC1Regs
0083d570   gEDMACC2Regs
0083d574   timer0Regs
0083d578   timer1Regs
0083d57c   timer2Regs
0083d580   timer3Regs
0083d584   timer4Regs
0083d588   timer5Regs
0083d58c   timer6Regs
0083d590   timer7Regs
0083d594   timer8Regs
0083d598   cycle_measure_overhead
0083d59c   DDR_Regs
0083d5a0   uiUsedDescRegionNum
0083d5a4   uiInitialHostFdqNum
0083d5a8   uiInitialMonoFdqNum
0083d5ac   uiUsedRxFlowNum
0083d5b0   uiQ662_pend_event_num
0083d5b4   intTSCL
0c000000   packetBuffer_SL2_Size0
0c010000   packetBuffer_SL2_Size1
0c020000   packetBuffer_SL2_Size2
0c030000   packetBuffer_SL2_Size3
0c040000   hostDescriptor_SL2
0c050000   monoDescriptor_SL2
0c060194   TCI6608_EVM_DDR_Init
0c0609d4   TCI6618_EVM_DDR_Init
0c0613d0   TCI6614_VDB_DDR_Init
0c061e14   TCI6614_Huawei_DDR_Init
0c062ab8   KeyStone_main_PLL_init
0c062e48   KeyStone_DDR_PLL_init
0c062fcc   KeyStone_PA_PLL_init
0c063098   lock_mem_prot_regs
0c063164   unlock_mem_prot_regs
0c06322c   KeyStone_XM_cfg
0c0632f4   KeyStone_L1_cfg
0c0633f0   KeyStone_L2_cfg
0c0635c4   edma_Init
0c063a34   Keystone_enable_PSC_module
0c063a98   Keystone_disable_PSC_module
0c063aec   Keystone_disable_PSC_Power_Domain
0c063b40   Reset_Timer
0c063b88   Timer_Init
0c063c50   Timer_One_Shot_Init
0c063d18   Watchdog_Timer_Init
0c063e14   Service_Watchdog
0c063e58   calc_cycle_measure_overhead
0c063eb0   TSC_init
0c063ecc   TSC_delay_ms
0c063f28   TSC_delay_us
0c063f70   Exception_cfg
0c0640cc   memory_protection_exception
0c0641b8   EXC_external
0c064398   EXC_internal
0c064484   EXC_nmi
0c0644a0   EXC_swgen
0c0646d8   KeyStone_QMSS_Linking_RAM_init
0c0647a8   KeyStone_QMSS_Descriptor_Regions_init
0c064b78   KeyStone_Host_Descriptor_Queues_init
0c064e28   KeyStone_Mono_Descriptor_Queues_init
0c064ff8   KeyStone_Copy_FDQ
0c0650c4   KeyStone_Qmss_Download_Firmware
0c065288   KeyStone_Qmss_Config_Acc_Channel
0c065478   KeyStone_Qmss_disable_Acc_Channel
0c065544   KeyStone_Qmss_config_Acc_Timer
0c0655b0   KeyStone_Qmss_Config_Reclaim_Queue
0c065618   KeyStone_pktDma_Global_Control
0c065680   KeyStone_pktDma_TxCh_config
0c0656d8   KeyStone_pktDma_configureRxFlow
0c0661f0   QueuePushCycleTest
0c066354   QueuePopCycleTest
0c066490   QueuePushToPopDelayTest
0c066568   QueuePushToAccumulationDelayTest
0c0667a0   QueuePushToPendInterruptDelayTest
0c06680c   QueueReclamationDelayTest
0c0668f0   PktDmaThroughput
0c067058   QueuePushPopTest
0c067294   DSPCoreAccessQueueTest
0c0672d0   QueuePendInterruptTest
0c067320   PktDmaThroughputTest
0c067374   PktDmaTest
0c067500   main
0c0676e0   __c6xabi_divd
0c0682c0   QMSS_init
0c068380   PktDMA_init
0c068498   checkQueues
0c068c20   _printfi
0c0690a0   QueueAccumulationISR
0c069430   QueuePendISR
0c069480   __c6xabi_divf
0c069820   fputs
0c06a42c   CP_INTC_Init_QM
0c06a538   QM_Interrupts_Init
0c06a860   free
0c06aae0   __c6xabi_divull
0c06b760   HOSTrename
0c06b900   __c6xabi_divul
0c06baa0   malloc
0c06bc40   setvbuf
0c06bf60   _auto_init_elf
0c06c0e0   Exeception_ISR
0c06c260   __c6xabi_frcmpyd_div
0c06c500   fputc
0c06c500   putc
0c06c8a0   fclose
0c06c9c0   HOSTlseek
0c06cac0   _wrt_ok
0c06cbc0   copy_in
0c06ccc0   HOSTopen
0c06ce80   atoi
0c06cf60   close
0c06d040   __TI_zero_init
0c06d120   exit
0c06d200   memset
0c06d2e0   HOSTread
0c06d3a0   HOSTunlink
0c06d460   HOSTwrite
0c06d520   __c6xabi_divu
0c06d520   __divu
0c06d5e0   _cleanup
0c06d6a0   _doflush
0c06d760   fseek
0c06d820   lseek
0c06d8e0   ltoa
0c06d9a0   write
0c06da60   HOSTclose
0c06db00   __c6xabi_frcmpyf_div
0c06de20   memcpy
0c06e000   __c6xabi_fixdu
0c06e080   __c6xabi_fixfu
0c06e100   __c6xabi_llshl
0c06e180   _c_int00
0c06e200   _minit
0c06e280   printf
0c06e300   readmsg
0c06e380   remove
0c06e380   unlink
0c06e400   __c6xabi_llshru
0c06e460   _subcull
0c06e4c0   memccpy
0c06e520   writemsg
0c06e578   C$$IO$$
0c06e580   __c6xabi_isinf
0c06e640   _args_main
0c06e680   puts
0c06e6e0   __c6xabi_negll
0c06e700   __tdeh_init
0c06e720   _nop
0c06e780   C$$EXIT
0c06e780   abort
0c06e7a0   __TI_decompress_none
0c06e7c0   __TI_decompress_rle24
0c06e7e0   linkingRAM1
0c07ace0   acc48_be
0c07c110   _ctypes_
0c07c908   __TI_Handler_Table_Base
0c07c914   __TI_Handler_Table_Limit
0c07c95c   __TI_CINIT_Base
0c07c9b4   __TI_CINIT_Limit
82000000   hostDescriptor_DDR
82040000   monoDescriptor_DDR
86060000   packetBuffer_DDR_Size0
86080000   packetBuffer_DDR_Size1
860c0000   packetBuffer_DDR_Size2
86140000   packetBuffer_DDR_Size3
ffffffff   __TI_pprof_out_hndl
ffffffff   __TI_prof_data_size
ffffffff   __TI_prof_data_start
ffffffff   __binit__
ffffffff   __c_args__
ffffffff   binit

[241 symbols]
